:100000000C9446050C94B1050C9494080C94B1051D
:100010000C94B1050C94B1050C94B1050C94B10588
:100020000C94B1050C94B1050C940D160C94B1050B
:100030000C94C0230C94B1050C94B1050C94B1053B
:100040000C94B1050C94B1050C94B1050C94B10558
:100050000C94B1050C9415240C94B1050C94B105C5
:100060000C94B1050C94B1050C94B1050C94B10538
:100070000C94B1050C94B1050C94B1050C94B10528
:100080000C94B1050C94B1050C94B1050C94B10518
:100090000C94B1050C94B105660A680A740A740AD6
:1000A000740A740A740A740A6A0A6C0A6E0A740A78
:1000B000740A680A760A740A740A300A660A740AAC
:1000C000740A6C0A740A740A740A740A740A740A48
:1000D0006E0A660A520A740A560A740A740A740A84
:1000E000320A6A0A740A740A600A740A740A740A80
:1000F000340A720A740A540A740A680A740A740A7E
:10010000640A580A740A5A0A6C0A740A740A740A4D
:10011000620A5C0A740A740A740A740A740A740A19
:10012000740A5E0A740A360A740A740A6A0A740A3D
:10013000740A720A740A740A740A740A740A740AD1
:10014000740A740A740A380A740A740A740A600A0F
:10015000740A740A740A740A740A740A740A740AAF
:10016000740A740A3A0A740A3C0A3E0A740A740A47
:10017000740A400A420A440A740A460A480A740A7F
:10018000740A740A700A4A0A740A4E0A4C0A500A1F
:10019000740A740A740A740A720A9A0AA80AB40AD7
:1001A000B40A8C0AB40AB40AB40AB40AB40AB40A87
:1001B000B40AB40AB40AB40AB40AB40AB40A8E0A75
:1001C000B40A900AB40AB40AB40AB40AAC0AB40A6B
:1001D000C30AAA0AB40AB40AB40AB40AB40AB40A2A
:1001E000B40AB40AB40AB40AB40AB40AB40A840A4F
:1001F000A00A920AA40AB40A940AB40A980AB40A91
:10020000A20A960AA60A9C0A9E0AB40AB40AB40A6A
:10021000B40AB40AB40AB40A860A880A8A0AAE0A78
:10022000B00AB40AB40AB40AB20A920BB00BBC0BFF
:10023000E00BF00BFC0B180C2F0C520C6F0CFA0C93
:10024000260DA00DD20DBC0DE30DF50DFD0D030E19
:10025000070E0D0E690E6B0E6D0E6F0EAF0E770E44
:10026000770E770E710E730E750E58147F14771576
:100270007F147715CB14EE14771545155415D7193F
:10028000D719011A011A5C1A871C871C871C901A3F
:10029000871C7B1B7B1B411C871C561C741C007B12
:1002A00046010203763A687F6577482B353B6978CB
:1002B000796439141E3C6A7A1D16041A1F3D6B06B8
:1002C0001B070821203E6C2C19091715223F6D11C0
:1002D000050B0A1C23406E7E100D182425416F3635
:1002E0000E0C122726427037380F33132D437175C9
:1002F00034322F2E44727C7D283031744573515036
:100300004A524D492A5466594F5C5F4C4B4E6263CA
:100310005A5D5E60295367585B565761475548429E
:10032000403E3C3A3B456843413F3D2B357E697A30
:10033000790078141E7C6A7B1D16041A1F7F6B06D9
:100340001B070821204D6C2C19091715224A6D1125
:10035000050B0A1C234C6E49100D182425516F36CD
:100360000E0C1227264F7037380F33132D5271752C
:1003700034502F2E4E72397D283065314B735464C2
:10038000586776012A773259745C5F6602036263AC
:100390005A5D5E60295344575B5655614746802934
:1003A0001E1F20212223242526272D2E2A2B141A16
:1003B0000815171C180C12132F302878041607097B
:1003C0000A0B0D0E0F33343579311D1B061905113B
:1003D000103637387D557A2C393A3B3C3D3E3F400C
:1003E00041424353475F6061565C5D5E57595A5BBB
:1003F00062634648324445677B7F65030102525081
:10040000514F68696A6B6C6D6E6F707172580049FC
:100410004C754A4D734B4E767C777E7466547225CC
:100420003032582000623A2530345820006525309B
:10043000325820002146554C4C21200021464621AF
:10044000200077253032582000214353335F463057
:10045000210A00214353335F5245414459210A0088
:10046000214353325F45305F4630210A0021435318
:10047000325F4630210A00214353325F4530210A62
:1004800000214353325F494E4954210A002143530E
:10049000315F45305F25303258210A000A5B4F56E4
:1004A000525D20004C2575200053257520000A4917
:1004B000443A253034582825642920004D6F75733F
:1004C000653A206E6F7420737570706F7274656416
:1004D0000A005225752000572575200057257520E4
:1004E00000572575200058257520004125752000EE
:1004F00049257520005B4348475D20000A5052544F
:100500003A25303258204953523A25303458200089
:100510005B5253545D20000A4552523A25303258FE
:10052000204953523A2530345820000A4B657962ED
:100530006F6172642073746172742E0A000A5553DD
:100540004220636F6E666967757265642E0A000AE1
:100550000A544D4B3A30616230656266382F4C5513
:1005600046410A0A003403490042004D0020005071
:1005700000430020006B006500790062006F00619D
:100580000072006400200063006F006E007600655A
:1005900000720074006500720000000E0374002EEB
:1005A000006D002E006B002E0000000403090409FA
:1005B000027400040100A0320904000001030101DB
:1005C00000092111010001224000070581030800F4
:1005D0000A090401000103000000092111010001C2
:1005E0002236000705820308000A090402000203FC
:1005F00000000009211101000122220007058303E8
:100600002000010705030320000109040300010382
:1006100000000009211101000122390007058403AF
:100620002000011201100100000008EDFEEE1B0188
:10063000000102000105010906A101050719E029D1
:10064000E7150025019508750181020508190129A2
:10065000059505750191029501750391010507192D
:100660000029F71500250195F875018102C00631B2
:10067000FF0974A1010975150026FF009520750872
:1006800081020976150026FF00952075089102C0A9
:1006900005010980A10185021601002637001A8193
:1006A000002AB700751095018100C0050C0901A151
:1006B000018503160100269C021A01002A9C02757E
:1006C0001095018100C005010906A101050719E087
:1006D00029E7150025019508750181029501750826
:1006E00081010508190129059505750191029501FA
:1006F000750391010507190029FF150026FF0095D4
:100700000675088100C0636F6E73756D65723A205F
:10071000253034580A0073797374656D3A2025309A
:1007200034580A000A002530325820006B6579627F
:100730006F6172643A20004C45443A2025303258AB
:100740000A00253032583A202530386225730A00D5
:10075000722F632030313233343536370A00646506
:100760006C5F6B65795F6269743A2063616E2774B0
:100770002064656C3A20253032580A006164645F59
:100780006B65795F6269743A2063616E27742061DA
:1007900064643A20253032580A003F00433E20006E
:1007A0004C25640A000A092D20436F6E736F6C6537
:1007B000202D0A4553432F713A09717569740A0057
:1007C0000A092D204D61676963202D0A643A096486
:1007D000656275670A783A096465627567206D61BC
:1007E000747269780A6B3A096465627567206B6593
:1007F00079626F6172640A6D3A0964656275672097
:100800006D6F7573650A763A0976657273696F6EF6
:100810000A733A097374617475730A633A09636FF2
:100820006E736F6C65206D6F64650A302D343A0904
:100830006C61796572302D34284631302D4634296B
:100840000A506175733A09626F6F746C6F61646509
:10085000720A6E3A094E4B524F0A003F004E4B52FD
:100860004F3A206F66660A004E4B524F3A206F6E29
:100870000A0074696D65725F72656164333228299C
:100880003A202530346C580A006B6579626F6172CA
:10089000645F6E6B726F3A2025580A006B6579624F
:1008A0006F6172645F69646C653A2025580A006B59
:1008B0006579626F6172645F70726F746F636F6C81
:1008C0003A2025580A00686F73745F6B6579626F10
:1008D0006172645F6C65647328293A2025580A00A8
:1008E0000A092D20537461747573202D0A00474343
:1008F000433A20352E342E30204156522D4C494259
:10090000433A20322E302E30204156525F4152431E
:10091000483A2061767235310A004F5054494F4EA3
:10092000533A204C5546412045585452414B455965
:1009300020434F4E534F4C4520434F4D4D414E4465
:10094000204E4B524F204B45594D41505F5345432C
:1009500054494F4E20424F4F544C4F414445525FF3
:1009600053495A450A004255494C443A2030616285
:100970003065626638202831313A35373A323320D3
:100980004D61792032322032303230290A00564906
:10099000443A2030784645454428742E6D2E6B2EFF
:1009A00029205049443A203078316265652849420F
:1009B0004D205043206B6579626F61726420636FD4
:1009C0006E76657274657229205645523A203078E9
:1009D000303030310A00444553433A20636F6E761D
:1009E0006572742049424D205043206B6579626FD7
:1009F00061726420746F205553420A000A092D2049
:100A000056657273696F6E202D0A000A6D6F7573DB
:100A1000653A206F66660A000A6D6F7573653A2045
:100A20006F6E0A000A6B6579626F6172643A206FBB
:100A300066660A000A6B6579626F6172643A206FBC
:100A40006E0A000A6D61747269783A206F66660AF0
:100A5000000A6D61747269783A206F6E0A000A6448
:100A6000656275673A206F6E0A000A646562756791
:100A70003A206F66660A000A0A626F6F746C6F61D3
:100A80006465722E2E2E2000433E200011241FBECE
:100A9000CFEFD0E2DEBFCDBF04B603FE49C08091E8
:100AA000880390918903A0918A03B0918B038730CA
:100AB000904BA740B04B09F03BC0109288031092B6
:100AC000890310928A0310928B0314BE0FB6F89418
:100AD000A89580916000886180936000109260000A
:100AE0000FBE1092010810920008E3E0F0E089E0E8
:100AF00080935700E491E695E370E150E33040F4D1
:100B0000F0E0EE0FFF1FE35DFE4F2081318102C058
:100B100020E030E280E090E0A2E0B0E0821B930BA6
:100B2000A109B109B595A79597958795FC010995F8
:100B300011E0A0E0B1E0EAE3FCE400E00BBF02C09A
:100B400007900D92A433B107D9F723E0A4E3B1E0F5
:100B500001C01D92A838B207E1F70E9473110C94EE
:100B60001B260C940000FF93EF93E0913401F09169
:100B70003501309709F00995EF91FF910895FC0137
:100B80008591803011F0EFDFFBCF0895FF27E0E281
:100B900030E247FF0CC0419597FF09C0EDE2609538
:100BA000709580959095611D711D811D911D27FF88
:100BB00002C0219530E350E2AA27660F771F881FF5
:100BC000991FAA1FA41710F0A41B63955A95A9F7A3
:100BD000AA3008F0A95FA05DAF93F3956115710588
:100BE0008105910541F7ED3211F4EF93F395F2177A
:100BF00018F43F93F395FBCF8F91B5DFFA95E1F7AA
:100C00000895E991F9918591803021F0853219F0AC
:100C1000AADFF9CF089520E0E89455915532C1F349
:100C2000503311F4689455915A3348F4505390F36B
:100C3000220F022E220F220F200D250FF4CF0EF4CB
:100C4000219589919991533619F3533729F15335E9
:100C500059F1BC0188279927E8945C3621F48991E1
:100C6000999168945591543639F446EF7EF077FFA8
:100C70000DC08FEF9FEF0AC055374AE039F0583565
:100C800040E121F0523642E009F00895FF93EF93DE
:100C90007DDFEF91FF91B7CFFF93EF93FC0181913F
:100CA0008030B9F360DFFBCFFF93EF9368DFF1CFC4
:100CB000DF93CF93CDB7DEB72596A3DFCF91DF913A
:100CC0000895282F80914101823071F08330B1F076
:100CD000813001F5E62FF0E038E0739FE00DF11D63
:100CE0001124E256FC4F13C0E62FF0E088E0789F15
:100CF000E00DF11D1124E25EFC4F09C0E62FF0E08B
:100D000038E0739FE00DF11D1124E256FD4FE49190
:100D1000E03819F480E090E008959E2F9077892FB5
:100D200090E034E0959587953A95E1F738E0239F78
:100D3000800D911D112444E0880F991F4A95E1F719
:100D4000EF709C012E0F311DF901EE0FFF1FE050D7
:100D5000F8498591949108955998519A0895519818
:100D6000599A08955898509A08955098589A089505
:100D70005198599A85E08A95F1F7000089B18695D6
:100D8000817008955098589A85E08A95F1F700008F
:100D900089B181700895CF93DF93EC010E94B8066A
:100DA000882341F0209731F085E08A95F1F7000023
:100DB0002197F4CFCE01DF91CF910895CF93DF93A8
:100DC000C2E3D0E00E94B806811108C0209731F03C
:100DD00085E08A95F1F700002197F4CFCE01DF91ED
:100DE000CF9108952E9826982F9827980E94AC06A8
:100DF0000E94B506E9E6F0E0808188608083E9988A
:100E00000895E19AE99A0E94AF060C94B506E99814
:100E10000E94AC060C94B506CF93DF932FB7F894DD
:100E2000C0910201D0910301CE01882781159F4F07
:100E300019F080E09FEF02C08FEF90E08C2B9D2B8C
:100E400090930301809302012FBFCE0199278F3F1A
:100E5000910581F5CD2FDD27C03FD10551F0CF3F62
:100E6000D10509F451C080917503C034D10599F4BE
:100E700007C08091750380FF33C08CE394E004C009
:100E800080FF2EC084E394E09F938F930E945806C6
:100E90000F900F9025C080FF37C0DF93CF938DE276
:100EA00094E09F938F930E9458060F900F900F909D
:100EB0000F902AC0CE018F6F019699F08091750333
:100EC00080FF0CC0DF93CF9385E294E09F938F93D4
:100ED0000E9458060F900F900F900F90CD2F01C0D9
:100EE000CFEF8091750380FF0CC01F92CF938EE1EE
:100EF00094E09F938F930E9458060F900F900F904D
:100F00000F908C2F90E002C08FEF9FEFDF91CF9179
:100F10000895CF93CAE1C15069F00E940C078F3F3A
:100F20002FEF920749F48FE99FE00197F1F700C096
:100F30000000F1CF8FEF9FEFCF91089510923A010B
:100F400010923901109238011092370180E090E838
:100F500090930101809300018FEF9FEF9093030125
:100F6000809302010895EF92FF920F931F93CF9306
:100F7000DF93082F109237018091750380FF0CC01A
:100F80001F920F9382E494E09F938F930E945806E0
:100F90000F900F900F900F90E9980E94AC060E945E
:100FA000B5068FE891E00197F1F700C000000E94BC
:100FB000B2068FE891E00197F1F700C000000E94AF
:100FC000AF0680E197E20E94CB06892B11F481E005
:100FD0007FC0C0E0D0E0FF24F39410E0EE24E3945F
:100FE00090E59A95F1F7C8010C2E02C0959587956A
:100FF0000A94E2F780FF04C0FE240E94B50602C0F6
:101000000E94B2060E94DE06892B11F482E060C0C5
:1010100082E390E00E94CB06892B11F483E058C054
:101020002196C830D105E1F680E58A95F1F7FF20D9
:1010300019F00E94B50602C00E94B2060E94DE06A8
:10104000892B11F484E044C082E390E00E94CB0637
:10105000892B11F485E03CC090E59A95F1F70E9448
:10106000B5060E94DE06892B11F486E031C082E3CA
:1010700090E00E94CB06892B19F0C2E3D0E009C0B2
:1010800087E026C0209759F025E02A95F1F7000067
:1010900021970E94C2068111F5CFCD2B11F488E073
:1010A00017C00E94DE06892B19F0C2E3D0E009C008
:1010B00089E00EC0209759F085E08A95F1F700008D
:1010C00021970E94C2068823A9F3CD2BB9F48AE0A8
:1010D00080933701809137018061809337010E94AE
:1010E000AF060E94B506E19AE99A8FEF9FEFDF9174
:1010F000CF911F910F91FF90EF9008958FEF9FEF89
:1011000090930301809302010E949E070E94AF0604
:101110000E94B506E19AE99ADF91CF911F910F9154
:10112000FF90EF900C9489071F920F920FB60F92C9
:1011300011242F933F934F935F938F939F9329B1E4
:101140009091760340910001509101014115504862
:1011500019F49093360111C080913601981769F007
:101160008F5F981751F08091000190910101909349
:101170003A018093390180E2DDC0809100019091B5
:10118000010196958795909301018093000120FFBE
:1011900009C0809100019091010190689093010134
:1011A000809300018091000190910101992780387E
:1011B000910509F4F9C0A8F48032910509F4F4C04E
:1011C00038F4009709F4F0C0409709F489C0A9C029
:1011D0008034910509F4E8C08035910509F480C098
:1011E000A0C0803C910539F150F48039910509F493
:1011F00077C0803A910509F094C084E64DC0803DE7
:10120000910509F46DC0803E910509F08AC0809176
:1012100000019091010190933A01809339018091EE
:10122000000190910101892F9927909301018093EA
:10123000000183E252C084E649990FC0882369F017
:1012400095E09A95F1F700008150F6CF882349F098
:1012500095E09A95F1F7000081504999F7CF8111F7
:10126000A3C0809100019091010190933A01809375
:1012700039018091000190910101892F9927909364
:1012800001018093000182E228C0882379F095E073
:101290009A95F1F700008150499BF7CF07C088234A
:1012A00049F095E09A95F1F7000081504999F7CF00
:1012B00081117AC0809100019091010190933A01CF
:1012C000809339018091000190910101892F992724
:1012D000909301018093000181E28093380133C033
:1012E000809100019091010190933A01809339011E
:1012F000809100019091010197FF02C080E101C03F
:1013000081E180933801809100019091010146E0D4
:10131000969587954A95E1F7909301018093000196
:1013200012C0809100019091010190933A01809345
:10133000390180E8809337018091370190E0982F40
:1013400088278F6F27C08091000190910101992714
:101350008F3F910511F480EFEDCF809103018F3F16
:1013600031F0809102018F3F11F080E4E3CF809152
:10137000020190910301982F882790930301809395
:1013800002012091000130910101809102019091B0
:101390000301822B909303018093020180E090E887
:1013A00090930101809300019F918F915F914F91E4
:1013B0003F912F910F900FBE0F901F901895CF93D4
:1013C000C82F8DEE0E94B3078A3F910521F48C2F20
:1013D000CF910C94B307CF910895E82FE695E69549
:1013E000E695EF70F0E0EB5BFE4F4081282F277011
:1013F00081E090E002C0880F991F2A95E2F7242F20
:1014000030E028233923232B11F4842B8083089583
:10141000E82FE695E695E695EF70F0E0EB5BFE4F82
:101420002081382F377081E090E002C0880F991F2B
:101430003A95E2F7422F50E048235923452B19F003
:101440008095822380830895482F50E0FA013397D6
:10145000E138F10508F048C0E45BFF4F0C94122618
:1014600087E108958FE108958CE5089580E6089559
:1014700082E6089587E2089583E508958FE208954E
:1014800089E3089587E308958FE3089587E4089535
:101490008FE4089586E508958EE508958FE7089511
:1014A00080E0089585E608958EE608958FE6089514
:1014B00080E3089588E3089580E4089588E408951A
:1014C00080E5089587E508958FE5089588E10895FA
:1014D00088E0089580E2089580E1089589E1089503
:1014E0008DE6089588E208958F7708958FE0089536
:1014F000CF93482F50E0FA017C97E834F105A0F52E
:10150000E353FF4F0C94122685E53EC08AE53CC0AC
:101510008BE53AC08CE538C08DE536C08EE534C029
:101520008FE532C080E630C081E62EC082E62CC056
:1015300083E62AC08FE628C081E726C082E724C060
:1015400084E722C085E720C087E71EC088E71CC06B
:101550008AE71AC08CE718C08FE716C080E714C06E
:1015600089E712C08BE710C0C82F1F928F938DE8B8
:1015700094E09F938F930E9458060F900F900F90C6
:101580000F908C2F01C084E5CF9108950F931F9386
:10159000CF93DF930E94EE238C010E940C07EC0195
:1015A000019631F4C8010E940624843F9140A8F3BB
:1015B000CE01DF91CF911F910F9108950E94F20605
:1015C0000C94010780917503816080937503E5E4B5
:1015D000F1E0119281E0E535F807D9F70895E82F99
:1015E000F0E0EB5BFE4F80810895E5E4F1E01192BD
:1015F00081E0E535F807D9F70895982F80914101EA
:10160000823048F092FB882780F990FD826091FD3E
:1016100084600C94DF090895CF93DF9380913701A4
:10162000882371F18091390190913A01209137011D
:101630009F938F931F922F9387E195E09F938F93B2
:101640000E9458068091370180750F900F900F907F
:101650000F900F900F9071F4809140018B3051F4F6
:1016600080E195E09F938F930E945806109240016D
:101670000F900F901092370110923A011092390199
:1016800080913801882309F440C0909138018091FD
:1016900044019817D1F18091390190913A0120913C
:1016A00038019F938F931F922F938CEF94E09F9319
:1016B0008F930E945806809144010F900F900F90D5
:1016C0000F900F900F9085FF04C09091380194FD0A
:1016D00006C084FF12C08091380185FF0EC0809142
:1016E00040018B3051F485EF94E09F938F930E94DB
:1016F0005806109240010F900F908091380180930E
:10170000440110923A0110923901E09140018E2F6C
:1017100090E08C30910508F026C3FC01EB5EFE4F93
:101720000C9412260E9407070E94EE239F938F932A
:1017300080EF94E09F938F930E945806109241018E
:1017400010924301109242010E94F50A0E948719EB
:101750000E94EE2390933F0180933E0181E065C09B
:1017600080913E0190913F010E940624893E934062
:1017700008F4F9C282E031C00E949E070E9401076E
:101780008FE99FE00197F1F700C000008FEF0E9402
:10179000B3078A3F910511F486E001C083E080938E
:1017A00040010E94EE239F938F938BEE94E09F93D2
:1017B0008F930E9458060F900F900F900F90D3C2F6
:1017C0000E9407072E98269A2F98279A0E94EE23A8
:1017D00090933F0180933E0184E080934001C3C217
:1017E00080913E0190913F010E940624853F9140E7
:1017F00008F4B9C285E0F1CF2E9826982F98279843
:101800000E949E070E9401070E94EE239F938F93E0
:1018100086EE94E09F938F930E9458060E94EE23D9
:1018200090933F0180933E0186E080934001C3CFB7
:101830000E940C07019609F496C20E94EE239F9322
:101840008F9381EE94E09F938F930E9458060E949D
:10185000EE2390933F0180933E0187E0E6CF809195
:101860003E0190913F010E940624853F914018F06F
:1018700089E0809340010E940C07019609F473C22D
:101880000E94EE239F938F938CED94E09F938F9310
:101890000E9458060E94EE2390933F0180933E01E0
:1018A00088E0C3CF80913E0190913F010E940624C1
:1018B000853F914018F089E0809340010E940C0719
:1018C000019609F450C20E94EE239F938F9387EDF7
:1018D00094E09F938F930E94580689E0A6CF82EFF1
:1018E0000E94B3078F3F2FEF920789F08A3F91053F
:1018F00089F40E94C60A8F3F3FEF930771F0D82FFB
:10190000CC270E94C60A9E01282BC90108C08FEF70
:101910009FEF05C08EEF9FEF02C080E090E09093B4
:101920004301809342010E94EE239F938F9382EDA7
:1019300094E09F938F930E9458068091420190916A
:1019400043010F900F900F900F90009711F482E0D9
:101950002BC08F3F3FEF930711F481E025C08E3FEE
:101960002FEF9207A1F38F3F910559F48CEB94E090
:101970009F938F930E945806109241010F900F90F1
:101980001FC09C0125583B4A2230310580F480EF6E
:101990000E94B3078A3F9105D1F683E00E94B30706
:1019A0008A3F9105A1F683E08093410109C0803B05
:1019B0003FEB9307C1F3882781159F4BA1F3C7CF56
:1019C000809141011F928F93809143018F93809169
:1019D00042018F938EEA94E09F938F930E94580662
:1019E0008AE0809340010F900F900F900F900F901E
:1019F0000F90B9C10E94EE239F938F9389EA94E0E0
:101A00009F938F930E9458060F900F900F900F9006
:101A100080914101823029F0833039F488EF0E94AF
:101A2000B3070E94FF160E94FD0A8BE080934001DD
:101A30000E94EE239F938F9384EA94E09F938F9369
:101A40000E9458060F900F900F900F900E940C0765
:101A50009C012F3F9FEF390709F485C121153105FE
:101A600019F02F3F310569F40E94F50A0E94871989
:101A70008CE994E09F938F930E9458060F900F90EB
:101A800072C190914101923009F44DC0933009F434
:101A9000CCC0913009F067C190913D01923099F02E
:101AA00028F4992341F09130C1F03AC0933081F18C
:101AB000943091F135C0803E21F0813E51F482E0B6
:101AC00005C081E003C08D31F9F483E080933D01CE
:101AD0004AC187FFE4C08F770EC1863309F118F43D
:101AE0008A3229F41DC08A3AD9F0863BC9F087FDB5
:101AF00005C00E94780A0E94ED0912C08F770E94EB
:101B0000780A0E94080A0CC08D3951F484E0DECFB7
:101B1000853431F485E5C3C0853411F485E5EBC027
:101B200010923D0120C1E0913C014E2F50E0493020
:101B3000510508F077C0FA01EF5DFE4F0C941226B4
:101B4000803E69F030F4833871F0843871F48FE7A7
:101B500057C0813E31F0803F41F481E05BC082E0BC
:101B600059C084E057C082E04BC087FF98C00E94F4
:101B7000F50A81E894E098C0893509F453C0803FA4
:101B800019F0823119F44EC083E044C010923C0138
:101B900087FD03C00E94240A82C00E94F50A87E7DD
:101BA00094E082C0833821F0843821F48FE738C074
:101BB00082E036C010923C0187FF9DC00E94F50A6A
:101BC0008DE694E071C010923C01823109F4CBC0E3
:101BD000893509F4C8C087FD03C00E94240A8BC060
:101BE0000E94F50A80E694E05FC0843121F0803FD6
:101BF000C9F486E00FC085E00DC0873799F480E016
:101C00000E94ED090FC0843169F487E003C0803F72
:101C100049F488E080933C01A6C0873719F480E03E
:101C20000E94080A10923C019EC090913B019130A5
:101C300009F443C038F0923009F463C0933009F4DA
:101C40007FC091C0863809F168F48338D1F020F460
:101C5000803819F582E06CC08438A9F08538E9F441
:101C60008BE01DC08C38A9F030F4873881F08B38B8
:101C7000A1F481E014C08D3871F0803F71F481E0EF
:101C800057C082E00CC08FE70AC086E008C080E041
:101C900006C089E004C08AE002C087FD03C00E943C
:101CA000ED0961C083E594E09F938F930E945806ED
:101CB0000F900F901092400156C0482F50E0FA014B
:101CC000E358F109EB30F10590F4E65DFE4F0C941A
:101CD000122682E045C08FE743C08BE041C086E01A
:101CE0003FC081E03DC089E03BC08AE039C010922E
:101CF0003B0187FD03C00E94080A35C089E494E0D7
:101D0000D3CF853279F030F4863171F08E3199F489
:101D100080E00BC0863221F0803F69F483E008C088
:101D20008DE503C083E501C081E50E94ED0905C092
:101D300080933B0118C00E94F50A10923B0113C02A
:101D40008E3169F020F48631B1F781E509C0853222
:101D500021F0863281F78DE503C083E501C080E084
:101D60000E94080AEACF81E0DF91CF910895809127
:101D7000790208950895CF93DF9300D01F92CDB7D5
:101D8000DEB720917F03243021F523E029839B8354
:101D90008A8382E08093E9008FEF9091E800815080
:101DA00095FD06C095ED9A95F1F700008111F5CFEC
:101DB0008091E80085FF0DC040E050E063E070E0F6
:101DC000CE0101960E9427138091E8008E778093C0
:101DD000E8000F900F900F90DF91CF910895CF936F
:101DE000DF9300D01F92CDB7DEB720917F03243060
:101DF00029F522E02983805891099B838A832093C7
:101E0000E9008FEF9091E800815095FD06C095EDB7
:101E10009A95F1F700008111F5CF8091E80085FFD8
:101E20000DC040E050E063E070E0CE0101960E94FA
:101E300027138091E8008E778093E8000F900F9031
:101E40000F90DF91CF910895CF93DF93EC019091A4
:101E50007F03943009F048C0809114018823D9F0A1
:101E6000809115018823B9F09093E90081E88150B1
:101E700049F09091E80095FD05C09AE29A95F1F736
:101E800000C0F5CF8091E80085FF2EC040E050E013
:101E900060E270E019C081E08093E90081E8815040
:101EA00059F09091E80095FD07C0EFE3F1E031971C
:101EB000F1F700C00000F3CF8091E80085FF14C067
:101EC00040E050E068E070E0CE010E94271380916E
:101ED000E8008E778093E80080E2FE01A9E5B2E099
:101EE00001900D928A95E1F7DF91CF910895CF93FC
:101EF000C0915701C1110BC00E94FA23643C794084
:101F00008105910520F081E080935701C1E08C2F7D
:101F1000CF910895FF920F931F93CF93DF93D82F04
:101F20000FB607FE83C080917F03843081F08091DB
:101F3000070190E001962091090130E0822393236C
:101F40002091080130E08217930709F0CBC00E946E
:101F5000770F811110C08091070190E001962091C8
:101F6000090130E0822393232091080130E0821799
:101F7000930709F0B7C00E94EE238C01C091E900DD
:101F8000CF709091EC00892F817090FD80E8C82B74
:101F900083E08093E90085E0F82E8091EB0085FDD9
:101FA00042C08091EB0080FF3EC08091EE0087FF31
:101FB0003AC08091080190910701981709F457C021
:101FC0009091E80095FF8CC0E0910501F091060129
:101FD000E80FF11D20818F5F909109018923809383
:101FE00008012093F1008091E80085FDE2CF809107
:101FF000E80080FFDECF8091E8008E778093E800D4
:10200000F0920401D6CF8091070190E001962091D3
:10201000090130E0822393232091080130E08217E8
:10202000930709F44AC0CF70C093E90040910701BB
:10203000842F90E001962091090130E082239323C0
:102040002091080130E08217930709F44EC0E09117
:102050000501F0910601E40FF11DD0838091070185
:102060008F5F909109018923809307013EC0809181
:10207000E80085FF35C0D093F10081E02091F200A7
:102080003091F300232B91F09091E80090FF0EC067
:102090009091E80095FF03C01092F100F9CF909164
:1020A000E8009E779093E800F0920401882309F4F9
:1020B000AACFCF70C093E90018C080910401882393
:1020C00009F4B1CF0E94EE239C018017910711F40F
:1020D000890163CF90910401915090930401F8CF4E
:1020E00080E0CCCF40910701B2CF80E0DF91CF916B
:1020F0001F910F91FF90089580917E03811104C07C
:102100000E948F150C94F115089510927E03089586
:10211000089542E061EC81E00E94A01242E061EC8F
:1021200082E00E94A01242E261EC83E00E94A012D1
:1021300042E261EC84E00C94A01280918103833030
:1021400009F455C030F4813071F0823009F48EC04A
:1021500008958A3009F47AC08B3009F460C0893060
:1021600009F09CC020C080918003813A09F096C09C
:102170008091E800877F8093E800809184039091AC
:102180008503892B21F460E289E592E003C060E0D9
:1021900080E090E070E00E9474138091E8008B77FB
:1021A0008093E800089580918003813209F076C021
:1021B0008091840390918503009719F0039709F0AB
:1021C0006DC08091E800877F8093E8008091E800EF
:1021D00082FD05C080917F038111F8CF5FC080919F
:1021E000F100809379028091E8008B7753C0809151
:1021F0008003813A09F052C0809184039091850355
:10220000892B09F04BC08091E800877F8093E8001C
:102210008091E80080FFFCCF8091140136C080914E
:1022200080038132D9F58091840390918503892BB5
:10223000A9F58091E800877F8093E8000E94D5127D
:1022400080918203809314010C94871980918003FC
:10225000813221F58091E800877F8093E8000E9419
:10226000D5128091830380937A0208958091800330
:10227000813AA1F48091E800877F8093E800809103
:10228000E80080FFFCCF80917A028093F10080917A
:10229000E8008E778093E8000C94D5120895809121
:1022A000790280935801109279020E94F50A0C94E9
:1022B00087190C944F110E949B2380917D038823E2
:1022C00029F00E94A82381110C948A1208950E947B
:1022D000BC23809158018093790208950C94671172
:1022E00008950C947011CF9384B7877F84BF0FB685
:1022F000F894A895809160008861809360001092A6
:1023000060000FBE90E080E80FB6F8948093610003
:10231000909361000FBE8AE89FE00E946E238AE0DE
:1023200091E00E94FA168FE495E00E94BF050E949A
:10233000DE0A0E94AE170E948F150E94F115789454
:102340000E94B01780917F03843029F00E94DF162D
:102350000E947011F7CF8DE395E00E94BF050E94A7
:1023600071118BE295E00E94BF05C3E080917F036D
:10237000853019F40E945B11F9CF0E94B4172091A7
:10238000E4003091E50080915501909156012817A5
:10239000390709F466C08091E4009091E5009093BC
:1023A0005601809355010E94770F882309F459C084
:1023B00080917F03843009F054C08091E9008F70D0
:1023C0002091EC00922F917020FD90E8892BC09312
:1023D000E9009091EB0090FF41C09091EE0097FFD3
:1023E0003DC09091080120910701291709F1209122
:1023F000E80025FF1DC0E0910501F0910601E90FFD
:10240000F11D30819F5F2091090192239093080173
:102410003093F1009091E80095FDE3CF9091E800B2
:1024200090FFDFCF9091E8009E779093E800D9CF9E
:102430002091F2003091F300232B81F09091E8007D
:1024400090FF0CC09091E80095FF03C01092F1003E
:10245000F9CF9091E8009E779093E8008F70809379
:10246000E9000E94DF1682CF292F33272330310560
:10247000C9F060F42130310581F02230310509F0D6
:1024800041C084E790E02FEA35E040C021323105B9
:10249000E1F02232310531F135C082E190E023E2F2
:1024A00036E034C099278130910549F028F0029731
:1024B00049F5E5E6F5E005C0EBEAF5E002C0EBE939
:1024C000F5E0849190E09F0121C064307105D0F463
:1024D000660F771FFB01EC5DFE4F2081318189E0A3
:1024E00090E014C06430710568F4FB01EE0FFF1F2B
:1024F000E45EFE4F20813181FB01E85EFE4F80816A
:1025000090E004C080E090E020E030E0FA01318308
:102510002083089584E189BD86E189BD09B400FE68
:10252000FDCF8091D8008F7D8093D8008091E0000E
:1025300082608093E0008091E00081FDFCCF0895EF
:10254000982F973068F59093E900981739F07091BB
:10255000EC002091ED005091F00003C0242F762F65
:1025600050E021FD02C09F5FECCF3091EB003E7F39
:102570003093EB003091ED003D7F3093ED003091D2
:10258000EB0031603093EB007093EC002093ED0092
:102590005093F0002091EE0027FDE5CF80E00895F4
:1025A0008F708093E90081E008958091800387FF18
:1025B00011C08091E80082FD05C080917F038111E8
:1025C000F8CF11C08091E8008B770BC080917F031A
:1025D000882349F08091E80080FFF8CF8091E800DF
:1025E0008E778093E80008952091E4003091E50013
:1025F00095E64091EC00842F817040FF23C08091CC
:10260000E80080FD1DC080917F03882399F085300C
:1026100099F08091EB0085FD11C04091E40050914C
:10262000E5002417350729F3915011F09A01E1CF05
:1026300084E0089582E0089583E0089581E008959C
:1026400080E008954091E80042FFDDCF0895CF92E9
:10265000DF92EF92FF920F931F93CF93DF93EC01E2
:102660008B017A010E94F412811135C0E114F1044A
:1026700039F0F70180819181081B190BC80FD91F10
:10268000C12CD12C0115110529F18091E80085FD9F
:1026900018C08091E8008E778093E8000E94DF16D2
:1026A000E114F10449F0F70180819181C80ED91E2F
:1026B000D182C08285E00FC00E94F412882311F3FA
:1026C0000AC089918093F10001501109FFEFCF1AE0
:1026D000DF0AD8CF80E0DF91CF911F910F91FF905B
:1026E000EF90DF90CF90089520918603309187037B
:1026F0002617370748F06115710539F42091E80075
:102700002E772093E80001C0B901FC0120E061159B
:10271000710569F180917F038823E1F18530E1F152
:102720008091E80083FD3AC08091E80082FD2CC0D2
:102730008091E80080FFEBCF8091F2009091F30050
:102740006115710551F08830910538F4219120937D
:10275000F100615071090196F3CF21E0089709F06B
:1027600020E08091E8008E778093E800D0CF21119F
:10277000D1CF0AC080917F03882361F0853061F05A
:102780008091E80083FD0AC08091E80082FFF2CFCB
:1027900080E0089582E0089583E0089581E008953F
:1027A00020918603309187032617370748F061157B
:1027B000710539F42091E8002E772093E80001C0DC
:1027C000B901FC0120E06115710581F180917F0361
:1027D000882309F43EC0853009F43DC08091E800AB
:1027E00083FD3BC08091E80082FD2DC08091E80010
:1027F00080FFE9CF8091F2009091F300611571059F
:1028000059F08830910540F424912093F1003196DD
:10281000615071090196F2CF21E0089709F020E09C
:102820008091E8008E778093E800CDCF2111CECF44
:102830000AC080917F03882361F0853061F0809128
:10284000E80083FD0AC08091E80082FFF2CF80E0BB
:10285000089582E0089583E0089581E008951F932C
:10286000CF93DF93CDB7DEB7AA970FB6F894DEBF4C
:102870000FBECDBFE0E8F3E08091F100819323E04B
:10288000E838F207C9F70E949D108091E80083FFA5
:102890002EC18091800390918103492F50E04A30EE
:1028A000510508F024C1FA01EB5CFE4F0C9412268E
:1028B000803821F0823809F01AC108C080917C0369
:1028C00090917D03992389F082600FC080918403E9
:1028D0008F70873008F00BC18093E9008091EB0086
:1028E00085FB882780F91092E9009091E800977F96
:1028F0009093E8008093F1001092F100D1C0282F4E
:102900002D7F09F0F4C0882319F0823061F0EFC008
:1029100080918203813009F0EAC0933009F080E0B1
:1029200080937D032EC08091820381112AC0809103
:1029300084038F702FEF280F263008F0D8C08093C3
:10294000E9002091EB0020FF1CC0933021F480911E
:10295000EB00806214C09091EB0090619093EB00CB
:1029600021E030E0A90102C0440F551F8A95E2F72B
:102970004093EA001092EA008091EB008860809317
:10298000EB001092E9008091E800877F8093E800D7
:102990000E94D512ACC08111AAC0109182031F778A
:1029A0008091E3008078812B8093E3008091E800A0
:1029B000877F8093E8000E94D5128091E80080FF15
:1029C000FCCF8091E30080688093E300111102C086
:1029D00082E001C083E080937F0389C08058823009
:1029E00008F085C080918203909183038C3D53E071
:1029F000950779F583E08A838AE289834FB7F89453
:102A0000DE01139620E03EE051E2E32FF0E0509328
:102A10005700E49120FF03C0E295EF703F5FEF7035
:102A20008E2F90E0EA3010F0C79601C0C0968D93CB
:102A30009D932F5F243149F74FBF8091E800877F36
:102A40008093E8006AE270E0CE0101960E94741360
:102A500016C06091840370918503AE014F5F5F4F94
:102A60000E943412BC01892B09F441C09091E80006
:102A7000977F9093E80089819A810E94D01380917A
:102A8000E8008B778093E80032C0803881F5809130
:102A9000E800877F8093E80080917B038093F100BA
:102AA0008091E8008E7772CF811121C080918203DE
:102AB0009091830399270297D4F48091E800877F4F
:102AC0008093E8008091820380937B030E94D5125B
:102AD00080917B03811106C08091E30087FD02C0D5
:102AE00081E001C084E080937F030E94891080917F
:102AF000E80083FF0AC08091E800877F8093E800A8
:102B00008091EB0080628093EB00AA960FB6F89458
:102B1000DEBF0FBECDBFDF91CF911F9108950E9400
:102B200000160E940816E0EEF0E08081816080834C
:102B3000E8EDF0E080818F77808319BCA7EDB0E0ED
:102B40008C918E7F8C9380818F7E808310927E0308
:102B500008950F931F93CF93DF930E9400160E9456
:102B60000816C8EDD0E088818F77888388818068D7
:102B7000888388818F7D8883E7EDF0E0808180689D
:102B8000808319BC10927F0310927B0310927D0307
:102B900010927C0300EE10E0F80180818B7F80832F
:102BA00088818160888342E060E080E00E94A0121A
:102BB000E1EEF0E080818E7F8083E2EEF0E08081C4
:102BC00081608083808188608083F80180818E7F2E
:102BD0008083888180618883DF91CF911F910F91DD
:102BE0000895E8EDF0E080818F7E8083E7EDF0E0EE
:102BF00080818160808381E080937E030C94A9159D
:102C0000E8EDF0E080818C7F80831092E2000895EF
:102C10001092DA001092E10008951F920F920FB601
:102C20000F9211240BB60F922F933F934F935F9304
:102C30006F937F938F939F93AF93BF93EF93FF9384
:102C40008091E10082FF0BC08091E20082FF07C00B
:102C50008091E1008B7F8093E1000E94DE168091DD
:102C6000DA0080FF1FC08091D80080FF1BC08091D8
:102C7000DA008E7F8093DA008091D90080FF0DC04A
:102C800084E189BD86E189BD09B400FEFDCF81E004
:102C900080937F030E947C1005C019BC10927F03B3
:102CA0000E9485108091E10080FF19C08091E200B0
:102CB00080FF15C08091E2008E7F8093E2008091BA
:102CC000E20080618093E2008091D800806280936E
:102CD000D80019BC85E080937F030E945911809130
:102CE000E10084FF30C08091E20084FF2CC084E1C9
:102CF00089BD86E189BD09B400FEFDCF8091D80071
:102D00008F7D8093D8008091E1008F7E8093E100D9
:102D10008091E2008F7E8093E2008091E2008160EA
:102D20008093E20080917B03882311F084E007C048
:102D30008091E30087FD02C081E001C083E08093C1
:102D40007F030E946E118091E10083FF24C0809177
:102D5000E20083FF20C08091E100877F8093E10043
:102D600082E080937F0310927B038091E1008E7F4D
:102D70008093E1008091E2008E7F8093E200809159
:102D8000E20080618093E20042E060E080E00E9427
:102D9000A0120E948810FF91EF91BF91AF919F9177
:102DA0008F917F916F915F914F913F912F910F90F4
:102DB0000BBE0F900FBE0F901F9018950895CF93E4
:102DC00080917F038823A1F0C091E900CF7090919A
:102DD000EC00892F817090FD80E8C82B1092E900EB
:102DE0008091E80083FD0E942F14CF70C093E9000A
:102DF000CF9108959093800280937F020895E0918F
:102E00007F02F0918002309721F00190F081E02D57
:102E1000099480E00895EF92FF920F931F93CF9350
:102E2000DF93E0917F02F09180023097B1F18C0145
:102E30000280F381E02D09958091750382FF2DC0FA
:102E400080FF04C08CE297E00E94BF05E80110E219
:102E500086E2E82E87E0F82E8091750380FF0BC094
:102E600088811F928F93FF92EF920E9458060F90D5
:102E70000F900F900F90115021961111EDCF80916E
:102E8000750380FF0AC084E297E0DF91CF911F9124
:102E90000F91FF90EF900C94BF05DF91CF911F91A0
:102EA0000F91FF90EF900895CF93DF9320917D02D3
:102EB00030917E022817390709F190937E028093A2
:102EC0007D02E0917F02F09180023097B9F0EC0131
:102ED0000680F781E02D09958091750382FF0EC071
:102EE00080FF0CC0DF93CF9386E197E09F938F9391
:102EF0000E9458060F900F900F900F90DF91CF9186
:102F00000895CF93DF9320917B0230917C022817A4
:102F1000390709F190937C0280937B02E0917F0254
:102F2000F09180023097B9F0EC010084F185E02D3A
:102F300009958091750382FF0EC080FF0CC0DF935E
:102F4000CF9386E097E09F938F930E9458060F904F
:102F50000F900F900F90DF91CF9108950C94571818
:102F60000E94E5230C94E20ABF92CF92DF92EF9287
:102F7000FF920F931F93CF93DF9300D000D01F9247
:102F8000CDB7DEB70E940C0B02E812E0F12C8F2DBA
:102F90000E94EF0AB82EF801C080C82639F4F394D5
:102FA0000F5F1F4FF0E1FF12F2CF30C08091750329
:102FB00081FD0E945818D12CEE24E3948C2D8E2193
:102FC000F9F0D982FA8291E08B2D8E2109F490E0FC
:102FD0009B830E94EE238160782F9D838C8349819F
:102FE0005A816B818D810E948E1849815A816B8133
:102FF0007C818D810E948623F80180818E258083CB
:10300000D394EE0CF8E0DF12D9CFC9CF8FEF8983CC
:103010008A831B820E94EE238160782F9D838C839C
:1030200049815A816B818D810E948E180E9485236F
:103030000E94FF1690918102891741F10E94FF16AC
:10304000809381029091750392FF0EC090FF0CC097
:103050001F928F9387E397E09F938F930E94580668
:103060000F900F900F900F90809181020F900F9012
:103070000F900F900F90DF91CF911F910F91FF90C4
:10308000EF90DF90CF90BF900C9497230F900F900C
:103090000F900F900F90DF91CF911F910F91FF90A4
:1030A000EF90DF90CF90BF9008950C94FD0A0895A3
:1030B000EF92FF920F931F93CF93DF9380E597E0FA
:1030C0000E94BF05C0E0D0E08CE2E82E81E0F82E3F
:1030D00002E417E08C2F0E94EF0A0E947323FF92F4
:1030E000EF921F928F93DF93CF931F930F930E94C2
:1030F000580621968DB79EB708960FB6F8949EBFD6
:103100000FBE8DBFC031D10529F7DF91CF911F913F
:103110000F91FF90EF90089508950895CF93DF9356
:10312000CDB7DEB72B970FB6F894DEBF0FBECDBF7D
:10313000942F4F83252F588769877A878B874A85F5
:103140005B85452B31F02F3F31F481E09F3F19F42F
:1031500003C081E001C080E080FD07C04F81588539
:1031600069857A858B850E948623DE01119686E02B
:10317000FD0111928A95E9F785E0FE0137960190ED
:103180000D928A95E1F749815A816B817C818D810D
:103190009E810E94811F2B960FB6F894DEBF0FBE52
:1031A000CDBFDF91CF910895CF93882309F465C0F7
:1031B000C82F8CEF8C0F813A20F080E58C0F8E3277
:1031C00048F48C2F0E94BF25811157C08C2F0E947C
:1031D00069220CC080E28C0F883058F4C77081E0FF
:1031E00001C0880FCA95EAF70E940E23CF910C9474
:1031F00048238BE58C0F833078F4C53A29F0C63A22
:1032000031F083E890E005C081E890E002C082E8F8
:1032100090E0CF910C94541788E58C0F873168F5B6
:10322000C83A89F0C93A91F0CA3A99F0CB3AA1F07C
:10323000CC3AA9F0CD3AB1F0CE3AB9F0CF3AC1F0DC
:1032400080E090E017C082EE90E014C089EE90E03C
:1032500011C08AEE90E00EC085EB90E00BC086EBCB
:1032600090E008C083EB90E005C084EB90E002C0E2
:1032700087EB90E0CF910C948117CF91089588232C
:1032800049F19CEF980F913A20F090E5980F9E320B
:1032900018F40E94B9220DC090E2980F983058F4AB
:1032A000877091E001C0990F8A95EAF7892F0E94F3
:1032B00014230C9448239BE5980F933020F480E06E
:1032C00090E00C945417885A873120F480E090E005
:1032D0000C9481170895882321F00E940E230C94EA
:1032E00048230895882321F00E9414230C94482336
:1032F00008950E942E230E94FD220E94482380E010
:1033000090E00E94541780E090E00C9481170E9496
:103310001E230C947919CF92DF92EF92FF920F93B4
:103320001F93CF93DF9300D000D01F92CDB7DEB7AD
:103330006C010E9499238111EAC285E0F601DE0149
:10334000119601900D928A95E1F7F6014081518125
:10335000238134812115310531F05F3F31F481E063
:103360004F3F19F403C081E001C080E080FDCFC26F
:10337000F601F280E580E2948FE0E82249835A83E7
:10338000FB82722F3D832C836F2D8D810E94E5215E
:103390008C010E94E4210E94D420E12FE295EF707D
:1033A0008E2F90E0FC01E15CFE4F0C941226812FE1
:1033B000807F1F70882311F01295107FFF2049F045
:1033C000112309F43BC2812F0E9421230E9448232C
:1033D00035C2802F0E943F19112309F498C2812F12
:1033E0000E9427230F900F900F900F900F90DF9166
:1033F000CF911F910F91FF90EF90DF90CF900C94A1
:103400004823812F807F1F70803211F01295107F2A
:10341000002319F0013009F12BC0FF20A9F0EE20A4
:1034200059F1F1E0812FEF1228C00F900F900F900B
:103430000F900F90DF91CF911F910F91FF90EF9020
:10344000DF90CF900C943123EE2021F021E0E216A2
:1034500009F45DC20E9434232DC0FF20E9F085E00D
:103460008E1508F454C20E940B23812329F022C038
:10347000FF20F1F0E11015C0812F0F900F900F90F9
:103480000F900F90DF91CF911F910F91FF90EF90D0
:10349000DF90CF900C946B1994E09E1508F437C21E
:1034A00009C0F601858180FFC9C18F708583E4CF93
:1034B000E110D7C1812F4AC1812F869586958370EF
:1034C00019F08130B9F023C2FF2019F0C8019370C0
:1034D00002C080E090E00F900F900F900F900F903F
:1034E000DF91CF911F910F91FF90EF90DF90CF90E0
:1034F0000C945417FF2019F0C801937002C080E0AB
:1035000090E00F900F900F900F900F90DF91CF9160
:103510001F910F91FF90EF90DF90CF900C94811747
:10352000812F837009F070C0F110F1C1202F229516
:1035300026952770220F220F602F6F70862F90E044
:10354000A0E0B0E06C017D01022E04C0CC0CDD1CBB
:10355000EE1CFF1C0A94D2F704FF12C08FE090E02B
:10356000A0E0B0E004C0880F991FAA1FBB1F2A95D6
:10357000D2F7BC01CD01609570958095909503C000
:1035800060E070E0CB011695169513701230B1F023
:1035900040F56C297D298E299F29113031F10F903A
:1035A0000F900F900F900F90DF91CF911F910F917F
:1035B000FF90EF90DF90CF900C94F9206C297D293B
:1035C0008E299F290F900F900F900F900F90DF91F1
:1035D000CF911F910F91FF90EF90DF90CF900C94BF
:1035E00013210E94F920C701B6010F900F900F9090
:1035F0000F900F90DF91CF911F910F91FF90EF905F
:10360000DF90CF900C94DF20FF2019F0812F817084
:1036100001C08695882309F47AC1202F229526952A
:103620002770220F220F602F6F70862F90E0A0E08E
:10363000B0E06C017D01022E04C0CC0CDD1CEE1C40
:10364000FF1C0A94D2F704FF12C08FE090E0A0E0C4
:10365000B0E004C0880F991FAA1FBB1F2A95D2F79C
:10366000BC01CD01609570958095909503C060E098
:1036700070E0CB011695169513701230B1F040F53D
:103680006C297D298E299F29113031F10F900F90DF
:103690000F900F900F90DF91CF911F910F91FF909E
:1036A000EF90DF90CF900C94C0216C297D298E295A
:1036B0009F290F900F900F900F900F90DF91CF9157
:1036C0001F910F91FF90EF90DF90CF900C94D2213B
:1036D0000E94C021C701B6010F900F900F900F906C
:1036E0000F90DF91CF911F910F91FF90EF90DF909E
:1036F000CF900C94AE21003FC1F128F480E4800FFC
:10370000803250F096C0023F09F45EC008F449C010
:10371000033F09F46CC08DC0F02FF071EF2E812FA4
:103720008F71FF2051F00E944721802FEE2019F069
:103730008295807FA2CE8F70A0CE0E946821802FBC
:10374000EE2019F08295807F01C08F700F900F904E
:103750000F900F900F90DF91CF911F910F91FF90DD
:10376000EF90DF90CF900C947219FF20A9F024E025
:103770002E1508F4CCC0812F8F710F900F900F90F1
:103780000F900F90DF91CF911F910F91FF90EF90CD
:10379000DF90CF900C948D2185E08E1508F4B7C092
:1037A000EACFFF2099F0812F8F710F900F900F902B
:1037B0000F900F90DF91CF911F910F91FF90EF909D
:1037C000DF90CF900C944721FF2069F3812F8F71F8
:1037D0000F900F900F900F900F90DF91CF911F914E
:1037E0000F91FF90EF90DF90CF900C946821FF2015
:1037F00089F0812F8F710F900F900F900F900F9085
:10380000DF91CF911F910F91FF90EF90DF90CF90BC
:103810000C9432210F900F900F900F900F90DF912A
:10382000CF911F910F91FF90EF90DF90CF900C946C
:103830002D21FF2099F0EE2009F4B5CF802F0F90B5
:103840000F900F900F900F90DF91CF911F910F91DC
:10385000FF90EF90DF90CF900C94D418EE2009F4F5
:10386000B5CF802F0F900F900F900F900F90DF919A
:10387000CF911F910F91FF90EF90DF90CF900C941C
:103880003F19412F4F70602FC6010E945A240F909C
:103890000F900F900F900F90DF91CF911F910F918C
:1038A000FF90EF90DF90CF900C942F2001112FC04C
:1038B000FF2069F10E9487199FEFE0E7F2E0915045
:1038C000E040F040E1F700C000000F900F900F9033
:1038D0000F900F90DF91CF911F910F91FF90EF907C
:1038E000DF90CF900C943B24412F4F70602FC60186
:1038F0000F900F900F900F900F90DF91CF911F912D
:103900000F91FF90EF90DF90CF900C945D240F907B
:103910000F900F900F900F90DF91CF911F910F910B
:10392000FF90EF90DF90CF9008951F93CF93DF9398
:1039300000D000D01F92CDB7DEB7942F4983252F3A
:103940005A836B837C838D834C815D81452B31F061
:103950002F3F31F481E09F3F19F403C081E001C0A3
:1039600080E0182F117080FD31C049815A816B8130
:103970007C818D810E94E521292F22952F702C308A
:1039800030F42A30A0F42250223030F022C02C3003
:10399000C9F02F30B9F01DC0853A28F48430C0F446
:1039A000823028F415C090E2980F983088F0883E55
:1039B00030F4803E68F48450813A58F409C0803F66
:1039C00041F406C093FB112710F903C010E001C0B9
:1039D00011E0812F0F900F900F900F900F90DF91BB
:1039E000CF911F910895CF93DF9300D000D01F9205
:1039F000CDB7DEB70F900F900F900F900F90DF9123
:103A0000CF910895CF93DF9300D000D000D0CDB7F1
:103A1000DEB726960FB6F894DEBF0FBECDBFDF919E
:103A2000CF9108951F93CF93DF93C091920216E038
:103A300080919302C81799F0D0E01C9FF0011D9F60
:103A4000F00D1124EC56FD4F40815181628173814C
:103A5000848195810E94021D2196C770E9CFDF9174
:103A6000CF911F9108954091C4025091C502609179
:103A7000C6027091C7028091C8029091C9020C944D
:103A8000021D0F931F93CF93DF938091C9028295FC
:103A90008F7009F05DC08091C602882309F458C078
:103AA00080919202109193026091C4027091C502BC
:103AB000C091C702D091C80291E06F3F09F090E039
:103AC000292F06E0811709F443C0209721F07F3F9A
:103AD00021F030E003C031E001C0322F90E030FD32
:103AE00034C0089FF001099FF00D1124DF01AC568E
:103AF000BD4F11963C911197371327C03C91361357
:103B000024C012963C91129731111FC013964D910B
:103B10005C9114974C1B5D0B483C5105B0F48091AF
:103B2000C9028F7080618093C902E756FD4F808182
:103B30008F708061808384EC92E00E948B19DF910A
:103B4000CF911F910F910C94121D01968770BACFDF
:103B5000DF91CF911F910F9108959F92AF92BF92E5
:103B6000CF92DF92EF92FF920F931F93CF93DF9349
:103B7000CDB7DEB761970FB6F894DEBF0FBECDBFED
:103B80008C0185E0F801DE011D9601900D928A9569
:103B9000E1F7F80140815181F280C380D480909197
:103BA000C4026091C5022091C7023091C80221155C
:103BB000310531F06F3F31F481E09F3F19F403C0CC
:103BC00081E001C080E0F82FF1709F2E80FD52C18E
:103BD00084ECA82E82E0B82EE090C602F601E21B2B
:103BE000F30BEE2009F4E8C08091C902E83CF1052E
:103BF00008F0A4C0282F207F09F053C0561313C02B
:103C0000491311C0EF2CF1100EC08F7080618093AA
:103C1000C9020E94331DC5010E948B198091C902FF
:103C2000F80185835BC1C114D10431F05F3F31F4E9
:103C300081E04F3F19F403C081E001C080E080FDC6
:103C400003C081E08F2502C080E090E0F82FF17082
:103C5000EF2E80FF1CC0809192022091930236E0EB
:103C6000821709F418C190E0389FF001399FF00DD8
:103C70001124EC56FD4F6181561306C06081461336
:103C800003C06281F61203C001968770E9CFEF2C62
:103C9000FF2009F423C18091C90281608093C90289
:103CA00062C0561306C0491304C0F11002C0F801E7
:103CB000A7C04D875E87FF867C2DD98AC88A6F2D65
:103CC00089890E94951C882399F1FF2089F1209110
:103CD000C902822F82958F7090E0029774F08091D4
:103CE000C4029091C50298878F831986DB86CA86A5
:103CF0002C87CE0107960E948B1986E0F801A4EC70
:103D0000B2E001900D928A95E1F70E94411D0E9458
:103D1000331D11C0561749F14D875E87FF867C2DF4
:103D2000D98AC88A6F2D89890E94951C81112CC05F
:103D3000C8010E948B19EE24E394D0C0282F207F65
:103D400049F77C2DD98AC88A6F2D89890E94F31C76
:103D500084EC92E00E948B1986E0F50111928A951D
:103D6000E9F70E94331DE12CB9C04913D5CFF110FA
:103D7000D3CFF8018583C8010E948B1986E0F50135
:103D800011928A95E9F7AAC0FF2091F22091C90209
:103D9000822F82958F7090E002970CF4AECF8091C5
:103DA000C4029091C5029A8389831B82DD82CC82F2
:103DB0002E83CE0101969FCFE83CF10508F04BC061
:103DC000EF2CFF2009F4B4CF561330C049132EC096
:103DD0002091C90220FD21C0822F82958F70482F2B
:103DE00050E041155105C9F0F80125834F305105C8
:103DF00041F08F5F982F9295907F822F8F70892B43
:103E00008583C8010E948B1986E0F801A4ECB2E01A
:103E100001900D928A95E1F72AC086E0F801A4ECA2
:103E2000B2E001900D928A95E1F758C04D875E8708
:103E3000FF867C2DD98AC88A6F2D89890E94951C9E
:103E400081115BCF8091C90281608093C902C80152
:103E50000E948B1943C07C2DD98AC88A6F2D89890D
:103E60000E94F31C86E0F50111928A95E9F70E9401
:103E7000331D34C0FF2009F45BCF4D875E87FF867A
:103E80007C2DD98AC88A6F2D89890E94951C882328
:103E900009F44ECF32CF7C2DD98AC88A6F2D8989FB
:103EA0000E94E521292F22952F70223028F49F703F
:103EB00039F0811105C00BC0243028F49F7049F4FB
:103EC000805E883020F0C8010E948B199E2CE92C5E
:103ED00005C0F8019581907F99F7F9CF8E2D6196F5
:103EE0000FB6F894DEBF0FBECDBFDF91CF911F910B
:103EF0000F91FF90EF90DF90CF90BF90AF909F9089
:103F000008951F93CF93DF93CDB7DEB72C970FB6ED
:103F1000F894DEBF0FBECDBF4F83588769877A877D
:103F20008B879C87CE0107960E94AD1D8823D1F018
:103F30009F8188852A853B85232B31F08F3F31F483
:103F400081E09F3F19F403C081E001C080E080FD63
:103F500047C04F81588569857A858B859C850E94ED
:103F6000021D3EC086E0FE013796DE0111960190EB
:103F70000D928A95E1F7FF81E8856A857B85611559
:103F8000710531F0EF3F31F481E0FF3F19F403C0D8
:103F900081E001C080E080FD23C02091930230E0E9
:103FA000C9010196877099274091920250E08417C9
:103FB0009507F1F1F983EA837D836C8396E0929F04
:103FC000D001939FB00D1124AC56BD4FFE01319628
:103FD00001900D929A95E1F7809393020E94121D31
:103FE00016E08091920290919302891771F1189FC7
:103FF000C00111248C569D4F0E94AD1D882329F1CC
:10400000E09192021E9FF0011124EC56FD4F408179
:10401000518162817381848195810E94021D80910A
:10402000920290E001968770992780939202D9CFEF
:104030000E9487191092930210929202E4ECF2E02F
:1040400086E0DF011D928A95E9F72C960FB6F89469
:10405000DEBF0FBECDBFDF91CF911F910895DF92DC
:10406000EF92FF920F931F93CF93DF93FC01892B65
:1040700009F488C0E12CF12CDD24D394EF012196C2
:104080008491853709F460C058F4843708F04EC035
:10409000843008F068C08130D1F0823071F172C094
:1040A000883709F45BC050F4863709F453C087376A
:1040B00009F068C08E2D0E941B2352C09CE7980F08
:1040C000903708F05FC08F770E943F194EC08F0174
:1040D0000E5F1F4FFE01849190E2980F983050F4CC
:1040E0008770FD2D01C0FF0F8A95EAF78F2F0E9480
:1040F000212315C00E94D41814C08F010E5F1F4FDA
:10410000FE01849190E2980F983068F48770FD2D3D
:1041100001C0FF0F8A95EAF78F2F0E9427230E9484
:104120004823E80122C00E943F19FBCFCF0102962D
:10413000FE01C491CC2361F0EFE9FFE03197F1F784
:1041400000C00000C150F6CFCF010296FE01F490EE
:10415000EC010BC00E940B23E82E07C00E941E2317
:104160000E94482302C00E94D4188F2D882341F05A
:10417000EFE9FFE03197F1F700C000008150F6CF82
:10418000FE017CCFDF91CF911F910F91FF90EF90B7
:10419000DF90089560934A0370934B0380934C0320
:1041A00090934D030C949623089560934E0370935F
:1041B0004F0380935003909351030C9495230F93D6
:1041C0001F9300914E0310914F03209150033091A3
:1041D0005103602B712B822B932B60934E037093B2
:1041E0004F0380935003909351031F910F910C94B0
:1041F00095230F931F9300914E0310914F0320912D
:1042000050033091510360237123822393236093E1
:104210004E0370934F0380935003909351031F916B
:104220000F910C9495230F931F9300914E031091BF
:104230004F0320915003309151036027712782274B
:10424000932760934E0370934F0380935003909392
:1042500051031F910F910C94952360E070E0CB0106
:104260000C94CA200F931F9341E050E060E070E08F
:104270008A019B0104C0000F111F221F331F8A9562
:10428000D2F7C901B8011F910F910C94CA200F9366
:104290001F9341E050E060E070E004C0440F551F00
:1042A000661F771F8A95D2F780914A0390914B033E
:1042B000A0914C03B0914D038A019B01082B192B4F
:1042C0002A2B3B2BC901B8011F910F910C94CA20D6
:1042D0000F931F9341E050E060E070E004C0440F92
:1042E000551F661F771F8A95D2F7409550956095A8
:1042F000709580914A0390914B03A0914C03B0912B
:104300004D038A019B01082319232A233B23C9015A
:10431000B8011F910F910C94CA200F931F9341E095
:1043200050E060E070E004C0440F551F661F771F27
:104330008A95D2F780914A0390914B03A0914C0348
:10434000B0914D038A019B01082719272A273B2793
:10435000C901B8011F910F910C94CA200F931F93AC
:1043600000914A0310914B0320914C0330914D036F
:10437000602B712B822B932B1F910F910C94CA20D1
:104380000F931F9300914A0310914B0320914C030C
:1043900030914D0360237123822393231F910F914A
:1043A0000C94CA200F931F9300914A0310914B0362
:1043B00020914C0330914D0360277127822793276A
:1043C0001F910F910C94CA2008958F929F92AF92E3
:1043D000BF92DF92EF92FF920F931F93CF93DF93E1
:1043E00000D000D01F92CDB7DEB76B837C838D8366
:1043F0008A018C819D81892B31F01F3F31F481E04E
:104400004F3F19F403C081E001C080E080FF03C08A
:1044100080E090E04DC08B818823D1F180904A03E9
:1044200090904B03A0904C03B0904D0380914E03AD
:1044300090914F03A0915003B0915103882A992A7B
:10444000AA2ABB2A8FE1E82EF12CD501C4010E2C3B
:1044500004C0B695A795979587950A94D2F780FDE5
:1044600006C081E0E81AF10880F7D12C07C0DE2CE5
:10447000B8018E2D0E946106019799F388E0189F7C
:10448000F0011124E653FD4FE00FF11DD08209C069
:1044900088E0189FF0011124E653FD4FE00FF11D55
:1044A000D08009831A8369817A818D2D0E946106EB
:1044B0000F900F900F900F900F90DF91CF911F9161
:1044C0000F91FF90EF90DF90BF90AF909F908F90F3
:1044D000089590911401992379F1909115019923F0
:1044E00059F1982F9695969596959F31A1F0E09168
:1044F0001601F0911701E90FF11D877021E030E0FE
:10450000A90102C0440F551F8A95E2F7CA019181A3
:10451000892B818308959091750390FF29C01F9284
:104520008F938CE797E09F938F930E9458060F908C
:104530000F900F900F900895209116013091170160
:10454000F90132969FEF40E05191851789F09F3F26
:1045500019F4511101C0942F4F5F4E31A9F79F3FBD
:1045600039F0F901E90FF11D97FDFA95828308955D
:10457000089590911401992381F190911501992347
:1045800061F1982F9695969596959F31A9F0E091B7
:104590001601F0911701E90FF11D877021E030E05D
:1045A000A90102C0440F551F8A95E2F7CA01809500
:1045B00091818923818308959091750390FF1CC098
:1045C0001F928F938EE597E09F938F930E945806DA
:1045D0000F900F900F900F900895E0911601F091B9
:1045E00017019F01225E3F4F9281891301C0128201
:1045F0003196E217F307C1F7089581E090E0E0916A
:104600001601F0911701E80FF91F10820196803210
:104610009105A9F70895809174030895909174030A
:10462000892B809374030895809590917403892356
:104630008093740308958093740308951092740313
:10464000089590917303892B809373030895809547
:1046500090917303892380937303089510927303D9
:104660000895809352030895109252030895809103
:10467000160190911701FC0131969C01205E3F4F7D
:1046800080E0919191118F5FE217F307D1F70895C0
:10469000E0911601F0911701809174038083E091FD
:1046A0001601F0911701908180917303892B80830B
:1046B00080915203882361F0E0911601F091170177
:1046C0009081892B80830E9437238111109252039D
:1046D00080911601909117010C940B17909335015E
:1046E0008093340108958295982F937344E0949FAA
:1046F000900111248C7C86958695282B822F8575B8
:10470000880F2A7A2695822B08950895CF93DF93F8
:1047100000D000D01F92CDB7DEB70F900F900F9052
:104720000F900F90DF91CF910895089508950C9404
:10473000551880E0089583B7817F8C6083BF83B76D
:10474000816083BF7894889583B78E7F83BF0895F7
:10475000CF930E948C180E940C0B0E948D18C0E011
:104760008C2F0E94EF0A811104C0CF5FC031C1F7C6
:1047700001C081E0CF9108950E94F50A0C94871939
:104780001F920F920FB60F9211248F939F93AF93A6
:10479000BF938091760390917703A0917803B091B5
:1047A00079034196A11DB11D809376039093770301
:1047B000A0937803B0937903BF91AF919F918F91AC
:1047C0000F900FBE0F901F90189582E084BD93E06C
:1047D00095BD9AEF97BD80936E0008952FB7F8941A
:1047E0008091760390917703A0917803B09179033B
:1047F0002FBF08952FB7F8946091760370917703D7
:1048000080917803909179032FBF08959C014FB751
:10481000F8948091760390917703A0917803B091FA
:1048200079034FBF821B930B089578941F920F92C8
:104830000FB60F9211248F939F93AF93BF938091E4
:10484000760390917703A0917803B0917903019654
:10485000A11DB11D8093760390937703A0937803F5
:10486000B0937903BF91AF919F918F910F900FBE3D
:104870000F901F9018950E948F15F89487E797E77F
:10488000909301088093000887E090EBDC0180930F
:10489000880390938903A0938A03B0938B039CE0D1
:1048A00088E10FB6F894A895809360000FBE9093AE
:1048B0006000FFCF80E090E008950895CF93C82F67
:1048C0001F928F9380EA97E09F938F930E945806E0
:1048D00081E090E0A0E0B0E0BC01CD0104C0660F33
:1048E000771F881F991FCA95D2F70E94D5200F9075
:1048F0000F900F900F90CF910C948719CF93873220
:10490000A8F58E3108F02BC1803109F49FC0F8F46E
:10491000873009F464C0A8F4863009F024C180917E
:104920007503817F8E7F8093750385EA97E00E94EF
:10493000BF0588E89AE00E94BF0581E080937A0372
:104940004CC08B30F1F18E3009F46CC00CC1863153
:1049500009F4B0C020F4813109F4EDC004C18931FB
:1049600009F491C08B3109F449C0FDC0883349F185
:1049700050F4893209F4F1C0853309F4EEC087326E
:1049800009F0F1C0EAC0833409F4E7C028F48A339F
:1049900008F4E9C08953E4C0883409F0E4C00E94F7
:1049A000871987E79AE00E94BF052FEF83ED90E318
:1049B000215080409040E1F700C000000E943B245D
:1049C0000CC080EC97E05CC08EE59AE00E94BF05C9
:1049D00080917503816080937503C1E0C9C08091A7
:1049E0007503C82FC17080FFEFCF8AE69AE00E945E
:1049F000BF0580917503817F8E7F3DC090917503C7
:104A000091FBCC27C0F981E0C827892FC0FB81F931
:104A100080937503CC2319F081E59AE027C083E4E5
:104A20009AE02EC09091750392FBCC27C0F981E0EB
:104A3000C827892FC0FB82F980937503CC2319F016
:104A400084E39AE013C084E29AE01AC0909175035F
:104A500093FBCC27C0F981E0C827892FC0FB83F9DD
:104A600080937503CC2351F088E19AE00E94BF0542
:104A7000809175038160809375037AC08BE09AE022
:104A80000E94BF05AACF8CEF99E00E94BF0586ED7A
:104A900099E00E94BF058EE899E00E94BF0586E676
:104AA00099E00E94BF058AE199E00E94BF058EEE61
:104AB00098E0E6CF80EE98E00E94BF050E94FF16C6
:104AC0001F928F9386EC98E09F938F930E945806D5
:104AD000809114011F928F938FEA98E09F938F9398
:104AE0000E94580680917A021F928F938CE998E079
:104AF0009F938F930E945806809115011F928F9368
:104B000089E898E09F938F930E9458060E94FA23A9
:104B10009F938F937F936F9382E798E09F938F93F8
:104B20000E9458068DB79EB746960FB6F8949EBF62
:104B30000FBE8DBF52CF0E948719C091150181E031
:104B4000C827C0931501CC2329F088E698E00E947D
:104B5000BF050EC08DE598E093CF80E001C08D5178
:104B60000E945E243ACF8BE598E00E94BF05C0E02A
:104B70008C2FCF91089580E008950C94BB25CF939E
:104B8000C82F80917A03882319F0813059F042C0F0
:104B9000E0911601F09117018081823261F0843436
:104BA000D9F509C0E0911601F09117018081823298
:104BB00011F0843461F48C2F0E94BD25811104C052
:104BC0008C2F0E947E2424C081E090E021C08C2F95
:104BD0000E94BB2581111BC0C43189F018F4CB3071
:104BE00029F010C0C93259F0C83361F485EA97E062
:104BF0000E94BF058CE997E00E94BF0508C0109293
:104C00007A030CC08AE997E00E94BF0507C081E0E3
:104C1000817006C010927A0380E002C080E0F8CF75
:104C2000CF910895EE0FFF1F0024001C0BBE0790CC
:0A4C3000F691E02D0994F894FFCFEF
:104C3A000080FFFF0559010000FFB70E240FBA0ECE
:104C4A00EF0EBB0E0101530340362239C606900609
:104C5A006E063506C105DA05F305130600001000D5
:044C6A00080004003A
:106800008800EA44E944E244040005000600070069
:10681000080009000A000B000C000D000E000F001C
:1068200010001100120013001400150016001700CC
:10683000180019001A001B001C001D001E001F007C
:10684000200021002200230024002500260027002C
:10685000280029002A002B002C002D002E002F00DC
:10686000300031003200330034003500360037008C
:10687000380039003A003B003C003D003E003F003C
:1068800040004100420043004400450046004700EC
:10689000480049004A004B004C004D004E004F009C
:1068A000500051005200530054005500560057004C
:1068B000580059005A005B005C005D005E005F00FC
:1068C0006000610062006300640065A185006700EC
:1068D000680069006A006B006C006D006E006F005C
:1068E0007000710072007300890087008A008B00BD
:1068F000E000E100E200E300E400E500E600E7007C
:106900000100010001000100EA4401000100E2442D
:106910000100010001000100460001004A004B0097
:10692000010001004700480001000100E9440100A6
:106930000100010001000100010001003A003B00DC
:106940003C003D003E003F0040004100420043004B
:10695000010035004C0039000100440045005200A0
:1069600049000100010050004F0029004D004E0079
:1069700051000100010001000100010001000100BF
:1069800001000100010001000100010001000100FF
:1069900001000100010001000100010001004D00A3
:1069A0004A004E004B0001000100010001000100FF
:1069B00001000100010001000100010001000100CF
:1069C00001000100010001000100010001000100BF
:1069D00001000100010001000100010001000100AF
:1069E0000100010001000100490001000100010057
:1069F000010001000100010001000100010001008F
:00000001FF
